:4000000080673030303030307e3030307e3030307e3030307e3030307e3030307e3030307d046b7e7e3030307d046e7e7d04167e7e3030307e3030307e3030307d03207e23
:4000400030303030303030303030303030303030303030303030303030303030303030307e3030307e303030711062e38770ef62e33841fefb50a64e62e33855f80055f9a5
:4000800000711062e00270ef62e338627105627505627905627d057c02c250005511173c11a6a0053f118ff8500157fa5511003c1103a00b08283f11187509008ff2711090
:4000c00043e32070ef62e000711062e00370ef62e2007c05cf8fff50107f3030303030303030303030303030303030303030303030303030303030303030303030303030d3
:4001000030303030303030303030303030303030303030303030303030303030303030303030303030303030303030303030303030303030303030303030303030303030bf
:4001400030303030303030303030303030303030889089008a618bf02300210022002700250026002b0029002a002f002d052e028c808d808e208f309ca09d419ea09f30e4
:4001800079fd7aa17b2078003f003d003e006038660063156500e640e700d600b000b100b200b333b433b500b600b87fb900ba10bb33bc33bd00be20ff202121652240245a
:4001c0000125152640282129352a402c292d162ec63c0e3dce3e4f61036900604062046733683363006600d100d300d000d200e1ffe200dfffde02dd00ff00000070ef62ab
:40020000000071106200006201ff70ef6203ff620200711062020062030070ef62010062040071106204006205ff70ef62078f620670711062060062070070ef62050062ea
:400240000800711062088062097f70ef620b7f620a807110620a00620b0070ef620900620c007110620c00620d0070ef620f00620e007110620e00620f0070ef620d006228
:400280001000711062100062110070ef621300621200711062120062130070ef621100621400711062140062150070ef621700621600711062160062170070ef6215007058
:4002c000ef7f7c02c97c01fd7f1070ef500067500157507c02e4500167500157b97c02e470ef207f380210084f56fc00d00456fc01182070ef62e30010082839ffa01f4fdb
:4003000048fc01a003711054fd18207509001008284f59fd610018207509008fd738fc7f7e43e1807f41e17f7f2901603f7f413ffe7f603d7f5d3e7f5d3f7f7110433e08d7
:4003400070ef7f7110413ef770ef7f21034f085d7b21fc2b00607b187f21fc4f085d792107480004b00a4178fe2b006079187f2700182b006079437801187f417bfc7f2105
:40038000034f085d9f21fc2b00609f5d8f21fc2b00608f187f11ff4b19004b4b08785bc005737480057373800108676767211f4f27fe202bfe5c18106464211f4f2bfe31fa
:4003c000202038ff29804b2980609c5b608c7f11ff4b19004b4b08785bc005737480057373800108676767211f4f27fe202bfe5c18106464211f4f2bfe31202038ff29801b
:400400004b2980436501609c4165fe5b608c7f419ffc418ffc7f7e43e1087f41e1f77f432f017f412ffe7f602d7f602e7f5d2e7f4f5d2e085d2f08412ffe71105d2d086276
:400440002d0070ef5d2c5d2e085200602e71105202602d70ef5201602f1838fd7ffffefcf8f0e0c00204081020408076127e4123fe438a20438b1071014070fe085d205dd1
:40048000227873d00376125314511253136221ff432301551200418bef418adf5115210fffc2082213a00b18110153135514ff80021868136e1468136e14182e151047165c
:4004c000ffa0177a16b0134127fe4123fe438a20438b1041e1fb41e1fe7e4f2103085d8b21fc2b0029f0608b498a01a00550065315187f418bfc7f53165115210f0107904a
:400500004f5d2a531250001212675512005d266221ff418bef418adf43230543270143e10443e1017f4127fe4123fe438a20438b100841e1fb41e1fe187f511521107f2687
:4005400015ef581351147f581351147f2615ef7f418afe9fd05515003907d00550078007390dc003500d11072c1501015c50016479bffd622600602a62253c010060297fb6
:400580001050057c0427201050027c042a7c041f20902590059019902e7f1050037c04da2010500d7c0550201050007c04f7207f1050037c037f207f1050f87c0359201003
:4005c00050037c034b207f1050047c0329207f104f38067c0580710141e0fe43e020711062087f6209ff70cf107c0338205311471120aff5107c033520539b3c9b10bfdf51
:40060000107c0338205311471120aff5107c033520539c3c9c02bfc7107c0338205311471120aff5107c033520539d50003a9dd03e5601035600008030107c033820531105
:40064000471120aff552015310551100540556040001015401107c03352053115205019b530e51113f0e770052003a9dcfcc519e54055604003d0400b0063d0501a0173de2
:400680000400b0063d0502a0133d0400b0063d0503a01b8027911990e680215f179f5f18a0511708511808912838fe800f5518105517105f99175f9a1890c45501008f1f2e
:4006c00038fa208fff085dd0085dd3085dd4085dd508511108511008510f08510e08510d08510c08510b08510a085109085108085107085106085105085104085103083c29
:400700000100b01b550101500008500a0850000808500008509b087c07ec38fa80081050ff7c03322018530318530418530518530618530718530818530918530a18530bd6
:4007400018530c18530d18530e18530f1853101853111860d51860d41860d31860d0187e107c03382053a551a521203920b00d107c033520539b5502018004559b057f711f
:40078000106208ff62097f10519970cf7c033220107c0338205311471120aff510519a7c033220107c0338205311471120aff57f107c053a203900aff8107c05475a112085
:4007c00053185f1711107c054c205f99175f9a187f104f1052fb0852fc207c03cf20207f7f62d000104f52fb60d58003104f52fc5310530f52fb531152fa80083f0f7bf85f
:400800001ff7003df800bff53df700bff0207f3030303030303030303030303030303030303030303030303030303030303030303030303030303030303030303030303007
:400840003030303030303030303030303030303030303030303030303030303030303030303030303030303030303030303030303030303030303030303030303030303078
:400880003030303030303030303030303030303030303030303030303030303030303030303030303030303030303030303030303030303030303030303030303030303038
:4008c00030303030303030303030303030303030303030303030303030303030303030303030303030303030303030303030303030303030303030303030303030303030f8
:4009000030303030303030303030303030303030303030303030303030303030303030303030303030303030303030303030303030303030303030303030303030303030b7
:020000040010ea
:020000040020da
:02000000eba370
:00000001ff
